:020000020000FC
:1000000018C01895189511C1189518951895189538
:100010001895189518951895189518951895010222
:100020000400000040404000000001010100000009
:10003000000022240FE50DBF02E00EBF00E806BD60
:1000400000E006BD379843E0A0E6BB27EEE1F0E014
:1000500002C005910D93E233E1F7D2D014D002E053
:1000600076D03327BAD06A30720510F42ED0F9CF8B
:100070006931720510F431D0F4CF6332720508F49F
:1000800034E609D0EECFE2E9F0E0332751E00BD0BF
:1000900008954040400052E0E0EAF0E004D00895C6
:1000A0002A2A2A555555C6E60591099304E628D013
:1000B000332339F4759079928590899204E620D0A3
:1000C00001C055D05A9579F7089552E0E4EDF0E07B
:1000D000EADF08952A5555552A2A52E0E4EEF0E069
:1000E000E2DF08952A2A5555552A52E0E4EFF0E060
:1000F000DADF08952A552A552A551197F1F7089500
:100100000F93BF93AF93B3E1A8E8F7DF0A95D9F750
:10011000AF91BF910F910895A32FBB275096AF9336
:10012000BF93B2E0AFEDE9DFBF91AF911197B9F79F
:1001300008950F93AF93BF930F930AE0E1DFE9F7C0
:100140000F910A95C9F7BF91AF910F9108950F9341
:10015000CF93DF93CAE00F9304E6D2DFCA95E1F7AD
:100160000F910A95B9F7DF91CF910F9108955F93A1
:100170005990688075908590AA24082D162D27D057
:1001800000950395C02EAA0C072D152D20D0B02E5A
:100190000C0D502F219759926882BEDF571004C072
:1001A000681002C05F910895952E990C9C1434F04C
:1001B0005C0DA0FC02C0539401C05A94B91454F3CE
:1001C0005B0DA1FC02C06394E5CF6A94E3CF011BF1
:1001D00018F4A39400950395089577276627BB9A92
:1001E000BC98B0E0A2E3C39A88DFC398B49BFECF6B
:1001F0006395721DB0E0A1E980DFB499F9CF08954D
:10020000F89403E0332427B3E0E6FF271191212B74
:100210000A95E1F727BB20BE28E020BF20E429BFD4
:100220002FBC2FEF2EBD789408950F930FB70F9327
:100230002F931F93EF93FF93FF274423C9F041307F
:1002400031F14230E1F13394032D033009F43324CA
:10025000ECE6E30D0081002331F028B3E0E6E30D86
:100260000081022B08BB2FBC1EE31EBD44272BC000
:10027000E6E6E30D10811EBD41E02FBC1EB5121154
:1002800003C01FEF1FBD1FC010E418BF1CC0ECE669
:10029000E30D2081222339F028B3E0E6E30D00814D
:1002A0000095022308BBE6E6E30D00811FEB42E068
:1002B0000E3B08F043E0101B1EBD2FBC04C043E002
:1002C0002FBC0FEF0EBDFF91EF911F912F910F915A
:0602D0000FBF0F9118950D
:00000001FF
